:1000000012C021C020C01FC01EC01DC03EC01BC0EA
:100010001AC019C018C017C016C015C014C013C02C
:1000200012C011C010C011241FBECFE5D4E0DEBF46
:10003000CDBF10E0A0E6B0E001C01D92A236B1072E
:10004000E1F71FD0ABC0DCCF8EB58B608EBD82EEEA
:1000500094E09BBD8ABD80E189BF7894089587B301
:10006000876087BB88B3887F88BB089580E0089548
:10007000882311F481E001C080E064E034D080E0A6
:100080000895EDDF19D0E0DFFFCF1F920F920FB67A
:100090000F9211248F939F93809160009091610043
:1000A000019690936100809360009F918F910F90D3
:1000B0000FBE0F901F90189580E487B983E086B932
:1000C000379A369A3699FECF84B195B1089597B193
:1000D0008F71907E892B87B9369A3699FECF24B1DD
:1000E00035B1C9010895BF92CF92DF92EF92FF928E
:1000F0000F931F93D82EB62ECC24EE24FF24870115
:100100000AC08D2DE4DFAC0160E070E0E40EF51E66
:10011000061F171FC394CB14A0F32B2D30E040E033
:1001200050E0C801B70118D0C9011F910F91FF908D
:10013000EF90DF90CF90BF900895882309F484E674
:1001400090E007C0E3ECF9E03197F1F700C0000060
:100150009F5F9817B8F30895A1E21A2EAA1BBB1B44
:10016000FD010DC0AA1FBB1FEE1FFF1FA217B30783
:10017000E407F50720F0A21BB30BE40BF50B661F99
:10018000771F881F991F1A9469F76095709580955D
:1001900090959B01AC01BD01CF010895F894FFCF6C
:00000001FF
